:10000000F89411240FEF0DBF00E10EBFA0E0B1E0A6
:10001000CCE0D1E0CA1BDB0B2196E2E4F1E02197B2
:1000200019F005900D92FBCFACE0B1E0CCE0D1E04F
:10003000CA1BDB0B2196219711F01D92FCCF02D039
:100040000C9402F0CF92DF92EF92FF920F931F93E6
:10005000CF93DF930F2EF8E3EF2EFF24F02D0F2E1A
:10006000F2E3CF2EDD24F02D0E94710080E091E0BC
:100070000E9492008FEF87BB83E081BBC1E0D0E09C
:10008000F701C0838D2F992787FD9A958370F6011C
:10009000808320E030E080E090E00196F5E7803357
:1000A0009F07DCF32F5F3F4F25303105A4F342E07B
:1000B000C030D40719F400E010E004C0C130D1050D
:1000C00009F48E010115110529F0CC0FDD1F88E020
:1000D00091E004C0D595C7958AE091E00E94920016
:1000E000CFCF109290008FE089B982E08BB988E180
:1000F0008AB986E0809395008F9A97988E98969A01
:1001000008955F9904C097985F9BFECF979A8CB132
:10011000992787FD909508958699FECF5D9BFCCF2A
:100120008CB90895CF93DF93EC018881882331F057
:1001300089910E948C0088818823D1F7DF91CF912B
:02014000089520
:0C0142006368617365720A002B002D00D9
:00000001FF
